:100000000C9434000C943E000C943E000C943E0082
:100010000C943E000C943E000C943E000C943E0068
:100020000C943E000C943E000C943E000C943E0058
:100030000C943E000C943E000C943E000C943E0048
:100040000C943E000C943E000C943E000C943E0038
:100050000C943E000C943E000C943E000C943E0028
:100060000C943E000C943E0011241FBECFEFD8E04C
:10007000DEBFCDBF0E9479020C9488020C94000070
:1000800081E084B985B90000000000000000000094
:10009000000015B800000000000000000000000093
:1000A0000000000000000000000000000000000050
:1000B000000085B900000000000000000000000002
:1000C00015B8000000000000000000000000000063
:1000D0000000000000000000000000000000000020
:1000E00085B900000000000000000000000015B805
:1000F0000000000000000000000000000000000000
:10010000000000000000000000000000000085B9B1
:1001100000000000000000000000000015B8000012
:1001200000000000000000000000000000000000CF
:1001300000000000000000000000000085B9000081
:100140000000000000000000000015B800000000E2
:10015000000000000000000000000000000000009F
:100160000000000000000000000085B90000000051
:10017000000000000000000015B8000000000000B2
:10018000000000000000000000000000000000006F
:10019000000000000000000085B900000000000021
:1001A00000000000000015B8000000000000000082
:1001B000000000000000000000000000000000003F
:1001C00000000000000085B90000000000000000F1
:1001D0000000000015B80000000000000000000052
:1001E000000000000000000000000000000000000F
:1001F0000000000085B900000000000000000000C1
:10020000000015B800000000000000000000000021
:1002100000000000000000000000000000000000DE
:10022000000085B900000000000000000000000090
:1002300015B80000000000000000000000000000F1
:1002400000000000000000000000000000000000AE
:1002500085B900000000000000000000000015B893
:10026000000000000000000000000000000000008E
:10027000000000000000000000000000000085B940
:1002800000000000000000000000000015B80000A1
:10029000000000000000000000000000000000005E
:1002A00000000000000000000000000085B9000010
:1002B0000000000000000000000015B80000000071
:1002C000000000000000000000000000000000002E
:1002D0000000000000000000000085B900000000E0
:1002E000000000000000000015B800000000000041
:1002F00000000000000000000000000000000000FE
:10030000000000000000000085B9000000000000AF
:1003100000000000000015B8000000000000000010
:1003200000000000000000000000000000000000CD
:1003300000000000000085B900000000000000007F
:100340000000000015B800000000000000000000E0
:10035000000000000000000000000000000000009D
:100360000000000085B9000000000000000000004F
:10037000000000000000000000000000000000007D
:10038000000015B8000000000000000000000000A0
:100390000000000085B9000000000000000000001F
:1003A000000000000000000000000000000000004D
:1003B000000015B800000000000000000000000070
:1003C0000000000085B900000000000000000000EF
:1003D000000000000000000000000000000000001D
:1003E000000015B800000000000000000000000040
:1003F0000000000085B900000000000000000000BF
:1004000000000000000000000000000000000000EC
:10041000000015B80000000000000000000000000F
:100420000000000085B9000000000000000000008E
:1004300000000000000000000000000000000000BC
:10044000000015B8000000000000000000000000DF
:100450000000000085B9000000000000000000005E
:10046000000000000000000000000000000000008C
:10047000000015B8000000000000000000000000AF
:100480000000000085B9000000000000000000002E
:10049000000000000000000000000000000000005C
:1004A000000015B80000000000000000000000007F
:1004B0000000000085B900000000000000000000FE
:1004C000000000000000000000000000000000002C
:1004D000000015B80000000000000000000000004F
:1004E00000000000E9EFF0E03197F1F700C00000F4
:1004F000C9CD389A91E088B1892788B92FE33DE0CA
:1005000083E0215030408040E1F700C00000F3CF8D
:04051000F894FFCF8D
:00000001FF
